:1000000000308A004828000083168510831285106E
:100010008316061283120612C7308C008C0B0E2832
:1000200000000000831685108312851483160612C3
:10003000831206167E281030840000080319282831
:10004000262800000000000000000000800B21288E
:1000500083288316051183120511831686108312D7
:1000600086108316051283120512C7308C008C0B84
:10007000372800000000831605118312051583162A
:10008000861083128614831605128312051688289B
:1000900084011F30830508308C008C1D57280730E1
:1000A0008101813084000008C0390F38800064006D
:1000B000813084000008C0390C04800083160610CB
:1000C0008312061483168113861183128615C73096
:1000D0008C008C0B692800000000831686118312A7
:1000E0008611831686168312861A7A28831681173C
:1000F00086288312831681178312042870308F009C
:10010000FA3090001B288F0B802883168312292831
:0A0110008316061083120610630028
:02400E00F03F81
:00000001FF
